:040000008031232800
:100008007A08200095006D08963E86002030031877
:10001800213087000108F100ED0A710E30390C38E3
:10002800F000F136F1367108250091007008930050
:1000380020006D085A3A0319ED010B1109008801D7
:100048008431092C00345234493446344634573408
:10005800413456344534CB0021005C082000CF00E1
:1000680021005B082000CE0021005B0A03195C0A0E
:100078000319003444284E0A03194F0A031960284B
:1000880020004F08CD004E08CC004D08BF004C089A
:10009800BE00C92080313F08CF003E08CE004C0882
:1000A800013EC90000304D3DCA004F06031D5E28C1
:1000B8004E08490603193F2821005B0820004C021E
:1000C800C90021005C0820004D3BCA004908013ED8
:1000D800D00000304A3D1A218031A42080313821D7
:1000E800803148082D21803121005B08FE3E200028
:1000F800D000FF3021005C3D20001A218031A4206F
:10010800803138218031210048082000D0072100A3
:1001180049082000D13D0030D23DD33D6908D007C1
:100128006A08D13D6B08D23D6C08D33D4B082D21A0
:100138004F082100DC0020004E082100DB000134BC
:10014800A001A101A201A301721CB2287608A00790
:100158007708A13D7808A23D7908A33DF635F70D4B
:10016800F80DF90DF536F40CF30CF20C750874045F
:1001780073047204031DA8282308F5002208F4005C
:100188002108F3002008F200080021004A08200096
:10019800C20021004B082000C300C401C501690842
:1001A800C2076A08C33D6B08C43D6C08C53D3F08DB
:1001B800C20701300318C3070318C4070318C5078B
:1001C8003F08C7003E08C600FF30C605C701C63550
:1001D800C70D4508B9004408B8004308B7004208ED
:1001E800B6004708BB004608BA000230BC004030E1
:1001F800BD008C31362480310038031D0829FF30BA
:100208002000BE00BF000800F20140308F3178277F
:10021800803173082000BF007208BE00FF303F0223
:10022800F83003193E02031C08000329D100D2014B
:10023800D30121005508F200F301F401F501200073
:100248005308F9005208F8005108F7005008F60062
:100258000800860087015008C03F5108C13F520876
:10026800C23F5308C33F08007508D3007408D20082
:100278007308D1007208D00008002000B001B10155
:10028800B201C130220097007D3021009D00F0307E
:100298009E000B302000A900B530A800A80B5229F9
:1002A800A90B522957292000AF01BC30A8005C29AE
:1002B8005D29A80B5B296029640021009D149D1805
:1002C80063291B082000A80021001C082000A900A1
:1002D800AA012808B0072908B13D2A08B23DAF0A8B
:1002E8000A302F02031C59292200970121001D10F2
:1002F80020003008F2003108F3003208F400F5015C
:100308003008A8003108A9003208AA00AA36A90CAA
:10031800A80C2808AB002908AC002A08AD00AE01DB
:1003280000302B07F600D8302C3DF7009F302D3DCC
:10033800F80000302E3DF900AC217408B2007308B3
:10034800B1007208B0003108A7003008A600080004
:10035800A101F51FBC29F209F309F409F509F20A0C
:100368000319F30A0319F40A0319F50AA101A10AEA
:10037800F91FCB29F609F709F809F909F60A03194B
:10038800F70A0319F80A0319F90A0130A106A201AC
:10039800A301A401A5017508740473047204031968
:1003A800012AA001A00AF51BDE29F235F30DF40D90
:1003B800F50DD629A235A30DA40DA50D7508790252
:1003C800031DF02974087802031DF02973087702C9
:1003D800031DF02972087602031CFB297208F60235
:1003E8007308F73B7408F83B7508F93B2214F53697
:1003F800F40CF30CF20CA00BDE29210803190F2AC8
:10040800A209A309A409A509A20A0319A30A0319A1
:10041800A40A0319A50A2508F5002408F4002308EE
:10042800F3002208F20008006C086B046A046904EF
:10043800031D0034BE30D2000130D300B601B7012D
:10044800B801B9015308BB005208BA001030BC000B
:100458004230BD008C313624823100380319003413
:100468002000460303194C2A4608043A03194C2A6B
:100478004608063A03194C2A46080B3A03194C2A2F
:1004880046080C3A03194C2A46080E3A031D6D2AF1
:100498004D08E900EA01EB01EC017A2282314C08AF
:1004A8003E04892282317A2282314B083E04892215
:1004B80082317A224A083E04E9003F08EA004008EF
:1004C800EB004108EC008E31DB268231003A031D37
:1004D800013410302000D2070318D30A0130530228
:1004E800FE300319520203180034222ABE006A089B
:1004F800BF006B08C0006C08C1004008C1003F087D
:10050800C0003E08BF00BE010800E9003F08EA003D
:100518004008EB004108EC0069080800B800B90180
:10052800BA01BD01BD0ABE01BF01C001C101B90ABE
:100538000319BA0A13303A02893003193902031829
:1005480000344108AE004008AD003F08AC003E084A
:10055800AB00AF01AF0A01308E3181268231BB007A
:10056800BC0138080319C52A4108B5004008B40081
:100578003F08B3003E08B2002930D2228231BB00C6
:10058800BC013B08C200C21B00343D080319CF2A36
:10059800C016BD019B2A421C01349B2AB600AB0140
:1005A800AC01AD01AE01AF01AF0A37308E31812603
:1005B8008231B700B71FE22A370808003719E02A46
:1005C8003508AE003408AD003308AC003208AB0083
:1005D800AF01AF0A36088E31812EA5010430A40080
:1005E800A301A201210019082000A0001330210056
:1005F800990020008C1221000C082000A100DE3098
:1006080021008C0020000C101230A600250875026D
:10061800031D182B24087402031D182B23087302CA
:10062800031D182B22087202031C2A2B64000314D2
:10063800260D2100970020002208F2022308F33B30
:100648002408F43B2508F53B63000A2BA603A536CE
:10065800A40CA30CA20CA61F0A2B21001710200023
:10066800210821008C0020002008210099000800A2
:10067800AA004038A4002308A5002208A6002108E3
:10068800A7002008A80003140530F200F301243065
:100698006023F900790DA900AA012A08243E8600E2
:1006A800870101088E31152683312000AA0A0630F9
:1006B8002A0203180800512BF500F8017208780285
:1006C8000318812B78087507F40086008701010854
:1006D800F600F701F33580307305F40076088039A9
:1006E80074060319792B0930F306F635F70A083032
:1006F8007702031C6E2BF80A622B73087F390800F7
:10070800F6007208F6077608013E860087010108A0
:100718002000A000A101A201A3012208A300210832
:10072800A2002008A100A0017608023E8600010868
:10073800A400A501A601A7012508A7002408A60072
:10074800A501A4017608033E86000108AB00AA01B2
:10075800A901A8012808A4042908A5042A08A604B0
:100768002B08A7042408A0042508A1042608A2042D
:100778002708A3047608860001082004F20021084F
:10078800F3002208F4002308F5000800A001A101E5
:10079800A201A30175087404730472040319002CE0
:1007A800A401A40AF51BDD2BF235F30DF40DF50DAC
:1007B800D52BA035A10DA20DA30D75087902031D37
:1007C800EF2B74087802031DEF2B73087702031DC3
:1007D800EF2B72087602031CFA2B7208F6027308D4
:1007E800F73B7408F83B7508F93B2014F536F40C10
:1007F800F30CF20CA40BDD2B2308F5002208F400FF
:100808002108F3002008F200080096308400203008
:1008180085005A30FE000030FF0184319D24843168
:10082800FA01E901EA01EB01EC01ED01C8308400AD
:10083800003085000F30FE000030FF0184319D2418
:100848000130FB002100FF30D700D800D900DA00C2
:10085800DB00DC00200088317228250824040319F5
:100868004C2CA801A80AA51B3C2CA435A50D362C98
:1008780025082702031D422C24082602031C482CA5
:100888002408A6022508A73BA536A40CA80B3C2CD7
:100898002708A5002608A400080022008C100C16C2
:1008A800240095121B30F200F20B582C22008C14F5
:1008B8001B30F200F20B5E2C22008C101B30F20071
:1008C800F20B642C240095160800F601F701721C3F
:1008D800712C7408F6077508F73DF435F50DF336F5
:1008E800F20C73087204031D6B2C7708F30076086A
:1008F800F2000800F301842C7408FF3A031D8E2CC3
:10090800FF308E3115268431F4008130F30A7302EA
:10091800031C802C74080800F400F200210056081B
:100928008A31A82284312100D60A5608031D0800FE
:10093800992C6400800101310130FE020030FF3B38
:100948007F087E04031900349E2CB601B701B80154
:10095800B901BA010230BB00BC01BD018C31362C93
:100968001530240092002A309500C0309400080009
:100978008B122500930121008C1220008C12080094
:10100000AB0032302B02031C1128750886008701C3
:101010000030C03FC13FC23F7608860081014131A8
:1010200081012B08F200053096268831AB00A6011D
:10103000A701A801AC012B08A02288312000A00044
:10104000A101A2012608A3002708A4002808A500E2
:101050002408A5002308A400A3012308A004240851
:10106000A1042508A2042008A6002108A700220840
:10107000A800AB0AAC0A03302C02031C1B2875081D
:10108000860087012608C03F2708C13F2808C23FC5
:10109000A901AA01AC012B08A02288312000A000E0
:1010A0002908A1002008A9002108AA00AB0AAC0A5F
:1010B00002302C02031C4B28760886008701290881
:1010C000C03F2A08C13F0800FF3015268831FF3095
:1010D00015268831FF3015268831F300FF3A031DAD
:1010E00008006A282100BA01BB01B301B401F03045
:1010F00099001F30980080308B00413022009D0005
:10110000CC3021008C0023008C0180302100950020
:1011100017100330A200AC30A100B330A000A00B28
:101120008F28A10B8F28A20B8F2864001530210077
:10113000A200DA30A1002030A000A00B9D28A10B56
:101140009D28A20B9D28A4288131412188312708A0
:101150002100BF00200026082100BE000E303F0203
:10116000113003193E02031CB8280A30C821883107
:10117000093021003F02C43003193E020318C3287E
:101180000B30C821883120000C142626883121001C
:10119000C200C208031DCF280130C821883187272B
:1011A0008831DB2688312100C200C208031DDB28FC
:1011B0000630C82188312100AE2788315623883176
:1011C00000380319FB282100BA0A0319BB0A430897
:1011D0001239031DDB282C08573A031DDB282D0884
:1011E000413A031DDB282E08563A031DDB28B30ABB
:1011F0000319B40ADB28210034083304031D032932
:101200000330C8218831210034082000A5002100C6
:1012100033082000A40040222A08A7002908A600BD
:1012200084313124883125082100BF0020002408A2
:101230002100BE00BA01BB01AE2788315623883198
:101240000038031941292100BA0A0319BB0A4308CF
:101250001239031D1C292C08573A031D1C292D087F
:10126000413A031D1C292E08563A031D1C29013042
:10127000BE020030BF3B3E0A03193F0A031944294E
:101280001C290930C821883121004108F300400899
:10129000F200FB2788310038031D51290730C8218F
:1012A00088312100B9019D294708B2004608B100E4
:1012B0004508B0004408AF004508A0004608A1005A
:1012C0004708A2002108A0002208A100A2012004D2
:1012D00003196F29B201B101FF30B000AF0030082F
:1012E000BD002F08BC003508F5003608F6003708A9
:1012F000F7003D08F9003C08F80039080F22883152
:101300002100B90A3C08B5073D08B63D0030B73D9D
:10131000B83D3C08A0003D08A100A201A30120089F
:10132000C4022108C53B2208C63B2308C73B470827
:10133000460445044404031D5429C4302000C80059
:10134000B53080312F2088310038031D9729F501F1
:10135000F601F701F801F90139080F228431A924B7
:101360008831BA220C10F501F4017530F3003030E9
:10137000F2008231F122883120000C1426268831B7
:101380002100C200C208031D032901300129C72919
:10139000F500F801F601750876020318FA290D30F8
:1013A000F4008330F3004530F200F20BD529F30B43
:1013B000D529F40BD5296400F70120008C160B30D9
:1013C000F300B530F200F20BE329F30BE329E8292F
:1013D00020008C120B30F300B530F200F20BEE2936
:1013E000F30BEE29F329F70A64307702031CDD2999
:1013F000F60ACB297E30F4001230F300D830F20028
:10140000F20B002AF30B002AF40B002AF80A05302D
:101410007802031CCA2920000C1063000D2A20004A
:10142000A00032302002031808002008F200053026
:1014300096268831A000A1017508F200210820023B
:10144000023EA82288312000A10A7608F50077081C
:10145000F600F70103302102031C1C2AA1017808C1
:10146000F20021082002043EA82288312000A10AAF
:101470007908F800F90102302102031808002F2A28
:10148000FF30A02288312000AF00B001B101B201CD
:101490008D278831FE30A022883120002B049C2724
:1014A00088318D278831FD30A022883120002B041F
:1014B0009C2788318D278831FC30A02220002B0406
:1014C000AF002C08B0002D08B1002E08B200F500C6
:1014D0003108F4003008F3002F08F200DE30F90084
:1014E000EC30F800E630F7006D30F6008031A420D3
:1014F00088310B307207AF000030733DB000003010
:10150000743DB1000030753DB200F200FF30A822FA
:10151000883120003108F200FE30A82288312000F6
:101520003008F200FD30A822883120002F08F20098
:10153000FC30A82220003208AA003108A9000800C7
:10154000F200230095017208910015141308080099
:10155000F300043023009500730891007208930093
:101560008B1355309600AA30960095148B17951C56
:101570000800B72A2000BF01BF0AC001C401D62756
:101580008831272BBF01C52AC601C101C201C30191
:101590004A08BA004B08BB00BC013C084302031DCB
:1015A000D72A3B084202031DD72A3A0841020318F2
:1015B000252B4308420441040319E12AC601642093
:1015C00088312000C5014508031DC6014608803A40
:1015D00003191A2B44080319F42AC403FF301526F3
:1015E00088312000C60AE62A7B086D060319E62A20
:1015F000FF30152688312000C400BA00BA36BA364A
:101600003A08BB007B08963EBC002030031821300E
:10161000BD003C0886003D0887003B088100FB0AAE
:101620007B085A3A0319FB01C60A2100540820001E
:10163000C400E62AC50A04304502031CE32AC10A95
:101640000319C20A0319C30AC82A1D268831473064
:10165000F5004A30F600400800208831C00A4908E9
:1016600048044704031D382B4B084A040319542B24
:101670004708B2004808B3004908B400B4268831CE
:101680002000BE00BE08031D482B0230C82188314F
:1016900020003F080319C42AD42488312000C60042
:1016A000C608031DC22A1D268431BC2C21004E0809
:1016B0002000CC0021004F082000CD00CE01CF013A
:1016C0006908CC076A08CD3D6B08CE3D6C08CF3D5C
:1016D000D001D101C401C50121004D0820004502FF
:1016E000031D762B21004C0820004402031800340F
:1016F0004F08B9004E08B8004D08B7004C08B600B6
:101700005108BB005008BA00BC01BC0A4830BD00FB
:10171000362488310038031900342000C808031922
:1017200000344808E53A0319202C48082E3A0319DA
:10173000202C0130BE020030BF3B3E0A03193F0A95
:10174000031D202C40080319C52B4808C600C701FB
:101750004808053A031DAF2BE530C600C701400815
:1017600086008701460881004F08A5278831013E81
:10177000BA000030513DBB000A30BC00400ABD0039
:101780003624883100380319003420004208031938
:10179000DA2B4F08A52788310B3EBA000030513DA7
:1017A000BB00BC01BC0A4208BD00362488310038A9
:1017B00003190034200043080319FB2B4F08A52709
:1017C00088311A3EBA000030513DBB000230BC00E7
:1017D0004830BD0036248831003803190034F20146
:1017E0004830782788312000430886008701720836
:1017F000C03F7308C13F4108031901344F08A527B2
:1018000088311C3EBA000030513DBB000430BC00A2
:101810004830BD0036248831003803190034F20105
:10182000483083318423883141088600870172085B
:10183000C03F7308C13F7408C23F7508C33F0134FD
:101840002030D0070318D10A5108023A5004031D72
:10185000322CD001D101CC0A0319CD0A0319CE0ACA
:101860000319CF0AC40A0319C50A6C2B21005A08B0
:1018700020003906031D4C2C210059082000380691
:10188000031D4C2C2100580820003706031D4C2C4A
:101890002100570820003606031D5A2C210053084A
:1018A00020003B02031D582C2100520820003A0260
:1018B00003189D2C2100570A0319580A0319590AC5
:1018C00003195A0A031D682C7A2CFF30152688311B
:1018D0002100D20A0319D30A520302300319530616
:1018E000031D652C1D268831FF302100DA00D90048
:1018F000D800D700200039082100DA00200038087D
:101900002100D900200037082100D8002000360827
:101910002100D70059082000B400210058082000F9
:10192000B300210057082000B200B42688310038E7
:10193000031900342100D201D30120003B0821000B
:101940005306031DA72C20003A0821005206031954
:10195000B02CD20A0319D30AFF30152688319D2CEA
:1019600020003C082100D2070318D30A2000BC0342
:101970003C08FF3A0319C62C3D0886008701FF305A
:101980001526883181002000BD0AB62C210053089D
:10199000023A5204031D01341D26FF302100DA00F3
:1019A000D900D800D7000134B4010430F300273047
:1019B000A22688310038031900342000B90113260B
:1019C00088312000B90A04303902031CDF2C0430AE
:1019D000F3002B30A22688310038031900340C3074
:1019E0002000B4077F3034020318012EB9013908F2
:1019F0002D3E860087011326883181002000B90A18
:101A000004303902031CF72C132688312000B30060
:101A1000132688310038031D00341326883100381E
:101A2000031D003413268831003A031D00340830AA
:101A30002000B4072D08663A031D042E2E086D3AC7
:101A4000031D042E2F08743A031D042E3008203A7B
:101A5000031D042E2100D401D40A13268831013A33
:101A6000031D003413268831003A031D0034200082
:101A7000B40AB40A132688312000B900132688312D
:101A8000003A031D00342000B90803190034210076
:101A90005408F20020003908962688312100D4002D
:101AA0002000B40AB40AB501B601B701B801B90102
:101AB000132688312000A800A701A601A50135083A
:101AC000A9003608AA003708AB003808AC002A087D
:101AD000A9002B08AA002C08AB00AC01250829049A
:101AE000B50026082A04B60027082B04B7002808EA
:101AF0002C04B800B90A04303902031C582D0430F4
:101B0000B4074530FA003808F5003708F400360805
:101B1000F3003508F2000230F235F30DF40DF50D47
:101B2000890B8C2D3508A5003608A6003708A700BC
:101B30003808A800A535A60DA70DA80D403025072B
:101B4000F6008A30263DF700F730273DF8000130D7
:101B5000283DF9008331CA2388317508B80074081C
:101B6000B7007308B6007208B500B901003038023A
:101B7000031DC02D00303702031DC02D0230360278
:101B8000031CC82DB90AB836B70CB60CB50CB62D67
:101B900008303902031800340830B100B2013908A6
:101BA0000319D92D3908B100B201FF30B107031C68
:101BB000B20321001508F0392000310421009500FE
:101BC00020003508003CFA00B901FF3015268831A5
:101BD0002000B90A06303902031CE52D0630B4078F
:101BE000FF3015268831083A031D0034FF301526D2
:101BF0008831003A031D00342000B40AB40A2100E1
:101C0000D403200034080800813033020318003464
:101C10003308B4072000B3033308FF3A0319F22C4A
:101C2000132688310A2EFF30152EF2007208240088
:101C30009100141C192E110808002000AB01AC0102
:101C4000AD01AE01AF01AF0A0C30812EC30184316A
:101C5000B42488310030C72788312000C501FF3007
:101C6000152688312000C50A14304502031C2F2E8A
:101C70008431512488312000AB01AC01AD01AE01AB
:101C8000AF01AF0A003081268831C500C30A1F307A
:101C9000430203180034450B382EAB01AC01AD01F3
:101CA000AE01AF01AF0A373081268831C500C51BB0
:101CB00000340030451D0130C40082319222883149
:101CC000003803190034AE01AD010230AC00AB01A5
:101CD000AF01AF0A103081268831C5004508031DC9
:101CE0000034AB01AC01AD01AE01AF01AF0A3B3036
:101CF00081268831C5004508031D00340130C727FF
:101D00000134B000FF30152620002E08A3002D0856
:101D1000A2002C08A1002B08A000300883313C232E
:101D2000883184317E242000B1000800F400F301E2
:101D300072087418F307F235F436F408031D982E70
:101D400073080800F500F3037308FF3A0319013420
:101D50007508F50A80310A008E31F40013268831A7
:101D60007406031D0034A32E3208AB003308AC0008
:101D70003408AD00AE010930AB35AC0DAD0DAE0D84
:101D8000890BBC2EAF01123081268831B500B51FFA
:101D9000CD2EEF30843190240034FF301526883169
:101DA0002000B500FF3A0319CD2E3508FE3A03197D
:101DB0000134EE30CA2EBE2788313630BA00BB015E
:101DC0000430BC005C30BD00362488310038031973
:101DD000003420005C08463A031DFA2E5D08413AA3
:101DE000031DFA2E5E08543A031DFA2E5F08313A9D
:101DF0000319FC2E8231182ABE2788310B30BA0015
:101E0000BB010D30BC005C30BD0036248831003889
:101E100003190034F2015C30782788317308023AE4
:101E20007204031D003420005E082100D500033039
:101E3000F2005C30782788317308CB007208CA0042
:101E40000630F2005C30782788317308CD007208C4
:101E5000CC000B30F2005C3078277308D100720898
:101E6000D00020006108F200F30121005108F500C4
:101E70005008F4008431692488317308CF00720857
:101E8000CE004A08CE074B08CF3DFF302000D400DB
:101E90000130D500D601D70121004C082000D80020
:101EA00021004D082000D900DA01DB010530D835CA
:101EB000D90DDA0DDB0D890B572F5808D4075908B7
:101EC000D53D5A08D63D5B08D73D0930D736D60CEC
:101ED000D50CD40C890B662F55082100C9002000B1
:101EE00054082100C8004E08C8074F08C93D0134F6
:101EF000F4007208F4077408860087017408013E34
:101F0000840085010008F3000108F20008002000A9
:101F1000E901EA01EB01EC010800AB003008AC007C
:101F20003108AD003208AE002D08AE002C08AD001F
:101F30002B08AC00AB010800AF002C08B0002D0846
:101F4000B1002E08B2002F080800B9004E08B800F2
:101F50004D08B7004C08B600500808003B082000A8
:101F6000BF0021003A082000BE00A430C000C430E9
:101F7000C100C330C200C030C30008006C08B90003
:101F80006B08B8006A08B7006908B6000800F200DC
:101F90000A30F300F40172080319D02FF301F401A1
:101FA00024001508F039730495000800F50180300D
:101FB000F2007508963EF300203003182130F4003B
:101FC000730886007408870072088100F50A5A3089
:101FD0007502031CD72F04309C001F309B000C306F
:101FE000250093009201910121008C12200095019F
:101FF0000B118B1608007308DC007208DB0001343B
:020000040001F9
:080000000000000000000000F8
:04000E00ACC9FFBDBD
:00000001FF
